BL51 BANKED LINKER/LOCATER V6.05                                                        07/31/2012  00:47:34  PAGE 1


BL51 BANKED LINKER/LOCATER V6.05, INVOKED BY:
D:\PROGRAM FILES\KEIL_51\C51\BIN\BL51.EXE task.obj, main.obj, zimo.obj TO xuanzhuan RAMSIZE (256)


MEMORY MODEL: SMALL


INPUT MODULES INCLUDED:
  task.obj (TASK)
  main.obj (MAIN)
  zimo.obj (ZIMO)
  D:\PROGRAM FILES\KEIL_51\C51\LIB\C51S.LIB (?C_STARTUP)
  D:\PROGRAM FILES\KEIL_51\C51\LIB\C51S.LIB (?C_INIT)


LINK MAP OF MODULE:  xuanzhuan (TASK)


            TYPE    BASE      LENGTH    RELOCATION   SEGMENT NAME
            -----------------------------------------------------

            * * * * * * *   D A T A   M E M O R Y   * * * * * * *
            REG     0000H     0008H     ABSOLUTE     "REG BANK 0"
            DATA    0008H     0006H     UNIT         ?DT?TASK
            DATA    000EH     0002H     UNIT         ?DT?ZIMO
                    0010H     0010H                  *** GAP ***
            BIT     0020H.0   0000H.1   UNIT         ?BI?TASK
            BIT     0020H.1   0000H.1   UNIT         ?BI?MAIN
                    0020H.2   0000H.6                *** GAP ***
            IDATA   0021H     0001H     UNIT         ?STACK

            * * * * * * *   C O D E   M E M O R Y   * * * * * * *
            CODE    0000H     0003H     ABSOLUTE     
            CODE    0003H     0003H     ABSOLUTE     
            CODE    0006H     16F0H     UNIT         ?CO?ZIMO
            CODE    16F6H     00D2H     UNIT         ?PR?OS_ALLRUN?TASK
            CODE    17C8H     008CH     UNIT         ?C_C51STARTUP
            CODE    1854H     0020H     UNIT         ?PR?_DELAY?TASK
            CODE    1874H     001FH     UNIT         ?PR?START?TASK
            CODE    1893H     0013H     UNIT         ?C_INITSEG
            CODE    18A6H     000BH     UNIT         ?PR?MAIN?MAIN
            CODE    18B1H     0007H     UNIT         ?PR?INIT?MAIN
            CODE    18B8H     0003H     UNIT         ?PR?INT0?TASK



OVERLAY MAP OF MODULE:   xuanzhuan (TASK)


SEGMENT
  +--> CALLED SEGMENT
---------------------
?C_C51STARTUP
  +--> ?PR?MAIN?MAIN
  +--> ?C_INITSEG

?PR?MAIN?MAIN
  +--> ?PR?INIT?MAIN
BL51 BANKED LINKER/LOCATER V6.05                                                      07/31/2012  00:47:34  PAGE 2


  +--> ?PR?START?TASK
  +--> ?PR?OS_ALLRUN?TASK

?PR?OS_ALLRUN?TASK
  +--> ?CO?ZIMO
  +--> ?PR?_DELAY?TASK



SYMBOL TABLE OF MODULE:  xuanzhuan (TASK)

  VALUE           TYPE          NAME
  ----------------------------------

  -------         MODULE        TASK
  C:0000H         SYMBOL        _ICE_DUMMY_
  D:0080H         PUBLIC        P0
  D:0090H         PUBLIC        P1
  D:00A0H         PUBLIC        P2
  D:00B0H         PUBLIC        P3
  D:00C0H         PUBLIC        P4
  D:00C8H         PUBLIC        P5
  D:00A8H         PUBLIC        IE
  C:1862H         PUBLIC        _delay
  C:16F6H         PUBLIC        OS_ALLRun
  D:00B8H         PUBLIC        IP
  D:00D8H         PUBLIC        CCON
  C:1874H         PUBLIC        start
  D:0098H         PUBLIC        SCON
  D:0088H         PUBLIC        TCON
  D:0008H         PUBLIC        ucNumRows
  B:0020H.0       PUBLIC        BIT_timeout
  D:000AH         PUBLIC        i
  D:000CH         PUBLIC        j
  D:00D0H         PUBLIC        PSW
  C:18B8H         PUBLIC        int0
  -------         PROC          L?0024
  -------         ENDPROC       L?0024
  -------         PROC          _DELAY
  D:0007H         SYMBOL        n
  -------         DO            
  D:0005H         SYMBOL        a
  D:0006H         SYMBOL        b
  -------         ENDDO         
  C:1862H         LINE#         37
  C:1862H         LINE#         38
  C:1862H         LINE#         40
  C:1868H         LINE#         41
  C:1868H         LINE#         42
  C:186AH         LINE#         43
  C:1870H         LINE#         44
  C:1873H         LINE#         45
  -------         ENDPROC       _DELAY
  -------         PROC          INT0
  C:18B8H         LINE#         47
  C:18B8H         LINE#         49
  C:18BAH         LINE#         50
BL51 BANKED LINKER/LOCATER V6.05                                                      07/31/2012  00:47:34  PAGE 3


  -------         ENDPROC       INT0
  -------         PROC          START
  C:1874H         LINE#         53
  C:1874H         LINE#         54
  C:1874H         LINE#         55
  C:1877H         LINE#         56
  C:187AH         LINE#         57
  C:187DH         LINE#         58
  C:1880H         LINE#         59
  C:1883H         LINE#         60
  C:1886H         LINE#         61
  C:1892H         LINE#         62
  -------         ENDPROC       START
  -------         PROC          OS_ALLRUN
  C:16F6H         LINE#         64
  C:16F6H         LINE#         65
  C:16F6H         LINE#         67
  C:16FCH         LINE#         68
  C:16FCH         LINE#         69
  C:16FEH         LINE#         71
  C:1706H         LINE#         72
  C:170FH         LINE#         73
  C:170FH         LINE#         74
  C:1714H         LINE#         75
  C:1714H         LINE#         76
  C:172FH         LINE#         77
  C:172FH         LINE#         78
  C:1746H         LINE#         79
  C:1754H         LINE#         80
  C:176FH         LINE#         81
  C:1776H         LINE#         82
  C:1776H         LINE#         83
  C:1779H         LINE#         84
  C:1782H         LINE#         85
  C:179DH         LINE#         86
  C:17A4H         LINE#         87
  C:17A4H         LINE#         88
  C:17A7H         LINE#         89
  C:17B0H         LINE#         90
  C:17B3H         LINE#         91
  C:17B6H         LINE#         92
  C:17B9H         LINE#         94
  C:17B9H         LINE#         96
  C:17B9H         LINE#         97
  C:17B9H         LINE#         98
  C:17C7H         LINE#         100
  C:17C7H         LINE#         101
  -------         ENDPROC       OS_ALLRUN
  -------         ENDMOD        TASK

  -------         MODULE        MAIN
  C:0000H         SYMBOL        _ICE_DUMMY_
  B:00A8H.7       PUBLIC        EA
  D:00A8H         PUBLIC        IE
  D:00B8H         PUBLIC        IP
  D:00D8H         PUBLIC        CCON
  C:18A6H         PUBLIC        main
BL51 BANKED LINKER/LOCATER V6.05                                                      07/31/2012  00:47:34  PAGE 4


  D:0098H         PUBLIC        SCON
  D:0088H         PUBLIC        TCON
  C:18B1H         PUBLIC        init
  B:0020H.1       PUBLIC        BIT_10MS
  B:0088H.0       PUBLIC        IT0
  B:00A8H.0       PUBLIC        EX0
  D:00D0H         PUBLIC        PSW
  -------         PROC          INIT
  C:18B1H         LINE#         24
  C:18B1H         LINE#         25
  C:18B1H         LINE#         29
  C:18B3H         LINE#         79
  C:18B5H         LINE#         80
  C:18B7H         LINE#         152
  -------         ENDPROC       INIT
  -------         PROC          MAIN
  C:18A6H         LINE#         169
  C:18A6H         LINE#         170
  C:18A6H         LINE#         171
  C:18A9H         LINE#         172
  C:18ACH         LINE#         174
  C:18ACH         LINE#         175
  C:18ACH         LINE#         176
  C:18AFH         LINE#         177
  -------         ENDPROC       MAIN
  -------         ENDMOD        MAIN

  -------         MODULE        ZIMO
  C:0000H         SYMBOL        _ICE_DUMMY_
  D:00A8H         PUBLIC        IE
  D:00B8H         PUBLIC        IP
  D:00D8H         PUBLIC        CCON
  D:000EH         PUBLIC        uiAllRows
  D:0098H         PUBLIC        SCON
  D:0088H         PUBLIC        TCON
  C:1056H         PUBLIC        love
  C:0006H         PUBLIC        zimo
  D:00D0H         PUBLIC        PSW
  -------         ENDMOD        ZIMO

Program Size: data=17.2 xdata=0 code=6331
LINK/LOCATE RUN COMPLETE.  0 WARNING(S),  0 ERROR(S)
